:030000000219FDE5
:03000B000200AA46
:03002B0002015976
:03005B000202E8B6
:030073000202D5B1
:1000800002030406080C10182030406080040608A3
:100090000C10182030406080A0C00003070F1F0D17
:1000A0000D0403060D0502030202C2AFC0D0C0E07A
:1000B000206214E5256009E473E525F4F58AD2622F
:1000C000D0E0D0D0D2AF3285268AC262E526F46075
:1000D0002AD0E0D0D0C295C294C293D2AF32C2959A
:1000E000C294C293206F0D20660A7405D5E0FDE529
:1000F0007BF45290D0E0D0D0D2AF32758A00C28D5E
:10010000D26201F401B9306805206602D29501B9C6
:10011000306805206602D29401B930680520660275
:10012000D29301B9D29230680A2066077403D5E0F1
:10013000FDD29501B9D29130680A2066077403D5C3
:10014000E0FDD29401B9D290D29230680A206607BD
:100150007403D5E0FDD29301B9C2AFC2AD53E6EF4F
:10016000C0D0C0E0D2D3D2AFC2CEE52A600720749F
:1001700049152A21BA7800790020742EE580307E56
:1001800001F430E70278FF53DACF207E0343DA2010
:10019000307E0343DA10C2D8C271E580307E01F4AC
:1001A00030E70279FFC3E89970CB306103752A40CC
:1001B000207403752A40885CD27020740DE52B6092
:1001C00004152B21CA43DA01C2D820700221DDA810
:1001D0005C206102C27020740221DB88227882B622
:1001E0000403852224C3E52594404002D26420CF35
:1001F0000AD0E0D0D043E610D2AD32C2CF053A7873
:1002000002E52A6005307402152AC3E55C940140BA
:1002100005755F004127756000756900E55F240181
:10022000F55F5003755FFF7982B7020D306E1DC315
:10023000E52294324016854C227982B7030E306E47
:100240000BC3E52294324004798E8722C3E52395BF
:1002500022600840041523415B0523D8CA0569E5DF
:100260006970021569D56A63756A017805C3E56925
:10027000956B4057C3E569956C50087801756A0322
:1002800002028FC3E569956D50057801756A01C357
:10029000E5629524401E7982B7040241C0206E14A5
:1002A000852462E569046003856B69756A017523BD
:1002B0003C0202CBE5622850057562FF41C0F56241
:1002C000E5620470067560FF7569FFD0E0D0D04329
:1002D000E610D2AD32C2AF53E67F7592FA7593FF46
:1002E000C260759104D2AF32C2AF53E6EFC2ADC067
:1002F000D0C0E0C0F0D2D3D2AFA8FBA9FCC2D830A6
:100300007102614F53DACF207E0343DA10307E034F
:1003100043DA20D271E580307E01F420E7026126C5
:1003200088278928A13453DACF207E0343DA20308E
:100330007E0343DA10C2D8C271307402A120780063
:10034000E580307E01F430E702A120885CA10853EB
:10035000DACF207E0343DA20307E0343DA10C27105
:10036000206102812853DACF207E0343DA10307EE9
:100370000343DA20C2D8D27188578958C3E895550B
:10038000F8E99556F97B007E087A00C3E8948CE979
:1003900094005005755B00811A882178A2E6A82197
:1003A0006055C3E894C8E994005008E4D2E4FB7AAD
:1003B0000A61F5C3E89468E994015008E4D2E3FBCC
:1003C0007A0F61F5C3E894D0E994025008E4D2E2D0
:1003D000FB7A1E61F5C3E894A0E994055008E4D2C5
:1003E000E1FB7A3C61F5C3E89498E994085008E48D
:1003F000D2E0FB7A787E00C3E89559FCE9955AFD76
:1004000030E70AECF42401FCEDF43400FD755B00E8
:10041000C3EC9AED9E5003755B018859895A855744
:10042000558558567802A108C3E89527F8E995281C
:10043000F9307C0281EC307B0281EC307A0281E57C
:10044000207502814BE9FDE8FC816AE9C313F9E8F4
:1004500013F830790281E5E9C313F9E813F830782D
:100460000281E5E9C313FDE813FC20612CC3EC9481
:0F0470001CED940240028181ED701EC3EC94C814
:10047F0050180529E52970021529C3E529940A505A
:10048F0002A120755C00D270A120E5296002152918
:10049F007400207F037896E624FAFEE43400FFC34D
:1004AF00EC9EFCED9FFD50067800790081ECC3ECCB
:1004BF0094FFED9400400678FF790081ECEC857293
:1004CF00F0A4C5F0A2F733F87900400302050878CD
:1004DF00FF7900020508E9C313F9E813F8307C0E21
:1004EF00E9600278FFC3E81338F8E43400F9C3E891
:1004FF0094FFE99400400278FF885CD2702061027B
:10050F00A120741FF4552F4BF52FC274EB7002D23C
:10051F0074752A40307403752A0A306102A13420A1
:10052F00740353DAFE207403752B20D0F0D0E0D083
:10053F00D0D2AD43E610327901020564790302058A
:10054F0064790A020564791E020564796402056400
:10055F0079C80205647817E4D5E0FDD8FAD9F622F8
:10056F007A147B7802058B7A107B8C02058B7A0DBF
:10057F007BB402058B7A0B7BC802058B7902E4D220
:10058F0091D5E0FDD294D5E0FDC294D5E0FDC291A6
:10059F00D5E0FDE920E002D29530E002D293E57379
:1005AF00D5E0FDE920E002C29530E002C2937496D7
:1005BF00D5E0FDD9C9EAF8D5E0FDD8FBDBBED29175
:1005CF0022C37C007D0075F00005F0EA33FAEB33AF
:1005DF00FB50F6EB13FBEA13FAC3E9FFE8FEE89AC8
:1005EF00F8E99BF95004EFF9EEF8B3EC33FCED3377
:1005FF00FDD5F0DFEDF9ECF822E889F08A20D2D4AE
:10060F00F8A9F07B0030F70B7BFFF42401F8E9F435
:10061F003400F9E88520F0A4ADF0F8E98520F0A4C6
:10062F00AFF0FEED2EF974003FFA7C04C3EA13FA23
:10063F00E913F9E813F8DCF48BF030F70AE8F42447
:10064F0001F8E9F43400F9E889F0C2D4F8A9F022EE
:10065F007882B604030206FEC3E55C9419401EE5DA
:10066F002D54067018206E3678057994E7146007BC
:10067F00780A1460027812C3E54198401F306E0962
:10068F008564627569FF756A01852224E4F544F576
:10069F0045F546F547F548C26E0206FED26E7994CF
:1006AF00E7147013E523F43333F913F8E954010415
:1006BF00F9E854FE0206F2E714147014E523F4333C
:1006CF003333F913F8E9540304F9E854FC0206FA3A
:1006DF00E523F433333333F913F8E954070404F9FA
:1006EF00E854F8C39440F8E99400F9884489452206
:1006FF00C3E54113F9E54013F8C3E54498F8E54520
:10070F0099F9500CC3E89480E994FF40160207361C
:10071F00C3E8947FE994005003020736787F79008D
:10072F00020736788079FF8849894A22E5492546AC
:10073F00F8E54A3547F9854A20E4300701F4354892
:10074F00FA30E709C3EA94F04015020774C3EA943C
:10075F000F500302077478FF79FF7A0F020774783E
:10076F000079007AF0C3E5249561500AC3740195AE
:10077F0024500B020792E54A20E70E020792E54A42
:10078F0030E706884689478A482278A5E6FAC3E506
:10079F004933F8E54A33F9D108E930E70BC3E89458
:1007AF0080E994FF4013E1CCC3E8947FE9940050B3
:1007BF0002E1CC787F7900E1CC788079FFE820E7FF
:1007CF0015C3E52398F84009C3E8940140030207D5
:1007DF00F378010207F3E8F424012523F84003021C
:1007EF0007F378FF884B2278A6E6FAA847A94812A4
:1007FF000608E930E70CC3E89401E994FF401602BC
:10080F000828C3E894FFE99400500302082878FFF2
:10081F007900020828780179FFE920E715C3E54B35
:10082F0098F84009C3E89401400302084F78010289
:10083F00084FE8F42401254BF8400302084F78FFD6
:10084F0088242278FFC26420693D206A12D264C3D3
:10085F00E541940A4009C3E52594405002C26479EA
:0E086F00A1E76023E541601F74FF8541F0841E
:10087D008539F0306A0375F005A4F8C5F06002788B
:10088D00FFC3E895645002A864886322C3E54094D1
:10089D0040E5419401E56350031401AA046002F59B
:1008AD0063227883E6F520120F2A75E8901205462B
:1008BD0075E890E5E820ECFBA8BDA9BE120FD47534
:1008CD006E55756F00C3740013FD7455606613FC8F
:1008DD0074552CFC74003DFDECFAEDFBC3E89AE970
:1008ED009B4014E56E2455F56EE56F3400F56FEA07
:1008FD002CFAEB3DFB80E5AE6EAF6FC3E56F13F9E0
:10090D00E56E13F8C3E913F9E813F87A03C3E91395
:10091D00F9E813F8DAF7AA201A7009756E00756FE9
:10092D00000209411AEA6008EE28FEEF39FFDAF8F5
:10093D008E6E8F6F2275E890227883E6FFE5E820B2
:10094D00ECF7A8BDA9BE0570C3E5709408405275BB
:10095D007000E9FA79A0E76044EA7007E571601B61
:10096D0002097CC3E895716010E5715006600C14A6
:10097D000209880460F9020988E571F571C3946D67
:10098D00401B7561C0C394044013756180C394040A
:10099D00400B756140C39404400375610075BB063F
:1009AD0022EFC39401601F7455601BC3E894FFE9E7
:1009BD0094035012C3E8956EE9956F5009E5616097
:1009CD000C15610209DAE561F460020561A861C3E5
:1009DD00E524985002A824C3E89562400AA862E570
:1009ED0062F4600385626188258826E570B407038B
:1009FD0075BB1022743279A787F0A4C5F0A2F73326
:100A0D00F8C3E895614002A861882288248825886A
:100A1D00268864227540007541F022C2AF75C8204A
:100A2D00A8CCA9CDAA3A30CF010A75C824D2AFAB54
:100A3D003BAC3C883B893CC3E89BF8E99C206908AA
:100A4D00F930670261344191AD3D8A3DF9EA9DFA75
:100A5D00600478FF79FFAE3EAF3F8B3E8C3FA83BE5
:100A6D00A93CC3E89EF8E99FF9C3E54113FBE540B6
:100A7D0013FAE82AF540E93BF54150067540FF753C
:100A8D0041FF41DBAA40AB41AC40AD417E047F024A
:100A9D00C3EB940440021E1FC3EB940840021E1FBB
:100AAD00C3ED13FDEC13FCDEF7C3EA9CFAEB9DFBE3
:100ABD00EF6009C3E913F9E813F8DFF7EA28FAEB59
:100ACD0039FB8A408B4150067BFF8B408B41C3EB3A
:100ADD0094025002D2673069047F0361067892E672
:100AED00FFC3E537948240110FC3E53794A0400151
:100AFD000FC3EF940640027F057E02E541C4540FFB
:100B0D00F9E541C454F0F8E540C4540F28F8C3E8A2
:100B1D009EFAE99400FB4009C3EA9402EB9400505D
:100B2D00047A02E4FB6180AA40AB41EBC4FEEAC447
:100B3D00540F4EFCC3EA9CFAEB9400FBC3E813C3BD
:100B4D0013F8EA28FAEB3400FB8A408B41C3EB948F
:100B5D00024002C2677802EBC4FE7B00EAC4540F68
:100B6D004EFAC3EA98FA4005C3940250027A02780D
:100B7D0092E6FF3060026180855192855293D2607A
:100B8D0043E680C3E49AF8E49BF9306702810CE8F0
:100B9D00FAE9FBD3E913FDE813FC88518952C3EF41
:100BAD0094036038EF20E00DE82CF8E93DF9ECFAFC
:100BBD00EDFB020BD5E828F8E939F9C3E82402F872
:100BCD00E93400F97AFE7BFFC3EF9403400E8A539C
:100BDD008B54884D894E8C4F8D508140885389544C
:100BED008A4D8B4E8C4F8D503069127553F0755464
:100BFD00FF754FF07550FF7551F07552FF8140E84C
:100C0D00FAD3E813FC8851C3EF94036020EF20E082
:100C1D0007E82CF8ECFA812CE8282402F87AFEC3B8
:100C2D00EF940340088A53884D8C4F814088538A36
:100C3D004D8C4FE568C3335002646BF5683060022C
:100C4D00814A753402D26043E680E52D5406603446
:100C5D00A840A941C3E913F9E813F8C3E913F9E86A
:0E0C6D0013F8306904E92440F9C2AF53E67F62
:100C7B00759100C3E498F594E499F595759104D2B8
:100C8B006043E680D2AF22D26575430075200030F9
:100C9B006C03752040020CB1D26575430075204082
:100CAB00306C0375200078017901206720E52D5405
:100CBB00066002C2657914E541C313700104F8C3E1
:100CCB00941440027814306904781B791B2060104F
:100CDB00E543600C306903D53404D26DA1539152B6
:100CEB000543E59B5440B52002A13D30690908C37B
:100CFB00E89940011881D820650A08C3E899400299
:100D0B0081B181D8C265C2AF53E67F759100306760
:100D1B00127594007595FE759104D26043E680D2EE
:100D2B00AF81B1AE40AF41C3E49EF594E49FF5951E
:100D3B00A122C3E5339401500281B130650281B128
:100D4B00D802A15181D8C26DC2AF53E67F75910015
:100D5B00855394855495759104854D92854E93D208
:100D6B006043E680D2AFE52D54066008206A020589
:100D7B0033020D8F306D0D206C0A20650715811520
:100D8B00810216072278003064053065027801E590
:100D9B003775F007A4F9E5F028F5F0E9A2F013A2F6
:100DAB00F113A2F213F537C394785003753778C358
:100DBB00E53795384008D266C295C294C29330602D
:100DCB0002A1C9854F92855093D26043E6802220C1
:100DDB007D16C2AF754202D291C292306202D2939B
:100DEB00D2AF759F11020FD1C2AF754202D291C221
:100DFB0090306202D295D2AF759F11020FD1307233
:100E0B0045207D22C2AF754203900135757B02C22E
:100E1B0093D290D292306204D294C129C291D2AFB4
:100E2B00759F01020FD1C2AF754203900135757BDF
:100E3B0002C295D292306204D294C149C291D2AF10
:100E4B00759F21020FD1207D17C2AF754203900110
:100E5B0010C293306202D294D2AF759F01020FD1B0
:100E6B00C2AF754203900110C295306202D294D288
:100E7B00AF759F21020FD1207D16C2AF754204D2F0
:100E8B0092C290306202D294D2AF759F21020FD1E1
:100E9B00C2AF754204D290D292C292306202D29407
:100EAB00D2AF759F01020FD1307243207D20C2AFAC
:100EBB00754205900124757B04C294D29130620473
:100ECB00D295C1D1C292D2AF759F11020FD1C2AFD1
:100EDB00754205900146757B01C294D29130620434
:100EEB00D293C1F1C290D2AF759F11020FD1207D69
:100EFB0017C2AF754205900106C294306202D295BB
:100F0B00D2AF759F11020FD1C2AF75420590011A76
:100F1B00C2943062EBD293D2AF759F11020FD120E6
:100F2B007D18C2AF754206D290D292C29130620246
:100F3B00D295D2AF759F01020FD1C2AF754206D2C7
:100F4B0092C291306202D293D2AF759F21020FD120
:100F5B00307245207D20C2AF754201900146757BF2
:100F6B0001C295D292306204D293E179C290D2AF92
:100F7B00759F21020FD1C2AF754201900124757B81
:100F8B0004C293D290D292306204D295E19BC2926A
:100F9B00D2AF759F01020FD1207D17C2AF754201F1
:100FAB0090011AC295306202D293D2AF759F210283
:100FBB000FD1C2AF754201900106C293306202D2CB
:100FCB0095D2AF759F01C26622900104757B00C25A
:100FDB0095C294C293D292D291D290C2622278805F
:100FEB0076070876070876010876040876FF0876F8
:100FFB00FF08760A087602087601087601788C7667
:10100B00010876000876B40876FF0876FF0876FFAD
:10101B000876030876FF0876010876FF0876250820
:10102B0076D00876780876C80876040876FF0876B6
:10103B000108760008767A08760A087601087601A8
:10104B000876000876FF087600227887E6FFC272E2
:10105B007888C27DE630E102D27DC27E7889E630A7
:0F106B00E102D27EC3EF94026008758E01D2734A
:10107A00021082758E00C273227880E61490008076
:10108A009378A5F67881E6149000809378A6F6788E
:10109A0086E61490008D9378A7F6789FE6F870019B
:1010AA0008C3E8941140027811E82828F56B256BEB
:1010BA00256B28F56C256B2828F56D7886E6F539B9
:1010CA00C394025003753902789CE67538FFB4025E
:1010DA00037538A0B4030375388278A3E614900028
:1010EA009A93F566120FD422227896E6FA7897E652
:1010FA00FB7888E6B40305C3EB940EFB307F047AD1
:10110A00007BFFC3EB9AFCC3948250027C82757207
:10111A00000572EC8572F0A4C3E5F0947D40F222DA
:10112A00D27F11F31205557A007B007C1012054B11
:10113A00E55C2AFA74003BFBDCF37C04C3EB13FB8B
:10114A00EA13FADCF7FEC27F11F322E5EF20E60389
:10115A007520000520903FFFE520146006901DFFD2
:10116A001460009304600375EF1253D9BF7581C0F0
:10117A0043FF8012054675EF0243B203E5B324022A
:10118A0020E70DF521E5E320E0068521B343E301DD
:10119A00120FD47580FF75A40075F19075D47F7510
:1011AA00908775A5BF75F2BF75D50075A60175E262
:1011BA0041120FD4E4F8F6D8FD756801120FE9124E
:1011CA00165E78988673753001C2AF12055F1205F4
:1011DA006F12055512057612055512057D12055531
:1011EA0012178112055F12055F12055AC2AF78FA0B
:1011FA0079FA308707D9FBD8F7021C0011551183F9
:10120A0011F211F378988673120FD47588107589C4
:10121A000275C82475910475D84075A82275B8025C
:10122A0075E690759B80759D0075D10E75BC5875D5
:10123A00BB0675BA1175E880120546D2AF1208AF1F
:10124A0075360053DACF207E0343DA20307E03431B
:10125A00DA1043DA01C2D8C27112055FD2617B0388
:10126A007A0CE55B70077A0CDB030211F61205555E
:10127A002070030211F6C270E55CC3940240E1E5F6
:10128A002F541F855E5DF55EB55DD5DAD5C2615313
:10129A00DACF207E0343DA20307E0343DA10C2D845
:1012AA00C27178A2E67008D274E52F54E0F52FC215
:1012BA007575290012055A307409C3E529940A4044
:1012CA0002D27512054B78023074027800C3E55CCD
:1012DA009840F0C2AF12056F12056F12056FD2AFB8
:1012EA0012055F754C0012054B788CE6C3940150C9
:1012FA00030213C6E530C3940150030213C62074D7
:10130A0035C3E55C94FF50030213C6C2AF120584CD
:10131A00D2AF12055AC3E55C940150EFC2AF120571
:10132A006F12055012056FD2AF12055AC3E55C94CD
:10133A00FF40E90218067F05D27F11F312055AC24F
:10134A00AFC27F11F3AE5CC3E55C947FD2AF407647
:10135A00120546C2AF120584D2AFDFDC312AC3EED2
:10136A0094057897F612055F1216A01217897F0A5C
:10137A00D27F11F312055AC2AFC27F11F3AE5CC31A
:10138A00E55C947FD2AF50E6120546C2AF12056FF4
:10139A0012055012056FD2AFDFD6312AEE24037838
:1013AA0096F612055F1216A01217B812055A11F313
:1013BA00C3E55C94FF50026108021806C3E55C9518
:1013CA004C4003855C4C12055A78017988E7B403CE
:1013DA00027805C3E55C98400241F0C2AF12058469
:1013EA00120584120584D2AF12055F753000E4F548
:1013FA0031F5320531E531F4703F0532789AE678F5
:10140A0019146012783214600D787D14600878FA25
:10141A00146003753200C3E53298401D120FD412CE
:10142A000546153275310078998673C2AF12058464
:10143A00D2AF7898867312055A120550E52A7005BC
:10144A0030740221F678012074027806C3E55C98AC
:10145A0040A112055AE52A70030211F6C2AF120F13
:0E146A00D4E4F522F523F524F525F526F567E3
:10147800D2AF7885E6C333F565E4F544F545F5461E
:10148800F547F548F570F52CF52DF53775700875A5
:10149800BB10120546120942E5E820ECFBA8BDA9DD
:1014A800BEE97001F8887112094675700875BB109D
:1014B8001155C2AF7561FF120A018522618522624A
:1014C800852263D2AF752201752401752501752621
:1014D80001856069756A017888E6B40307C27D30C2
:1014E8007602D27DD268D269753300120F2A120FA4
:1014F8005B120A21120A28120A21120A28120A214A
:10150800120CA312065F120D90120DDA120A28129D
:101518000C92306E031206FF2067031208523067E0
:1015280003120899120D90120E09120A28120CA320
:10153800306E0312073B120D90120E82120A281207
:101548000C92306E03120799120D90120EB3120A04
:1015580028120CA3306E031207F6120D90120F2AF0
:10156800120A28120942120C92120D90120F5B12E5
:101578000946120A2830692C856461856462856091
:1015880069756A0179187A0CC3E533994009C2690B
:10159800D26A8A350215ACC3E55C94014003021592
:1015A8000802160F306A1D206C1AE535147006C241
:1015B8006AD26BA108F535C3E55C940140030215B6
:1015C8000802160F753600C3E55F9401400985646B
:1015D80062856069756A0178FA79A4E76002780320
:1015E800C3E55F985021307404E52A601A78F0301A
:1015F8006C058564617820C3E541985002A108050F
:1016080036E55C6002C112753600C2AF120FD4789D
:1016180087E6FE760211557887EEF6E4F522F52383
:10162800F524F525F526F565752C00752D00D2AF46
:1016380012055A120FD478A4E66006C292C291C26B
:1016480090307406E52A700221F6788DE6C394017D
:10165800400241CD61F8901A0D78201216E2E5207B
:10166800B4A50CA31216E2E520B45A0302168012A0
:101678000FE91216A002169F901A0378807B0A12AF
:1016880016E2A308DBF9901A0F788C7B191216E280
:10169800A308DBF9901A2822C2AF1217211216FBF1
:1016A800901A00740E1216E7A374061216E7A374B4
:1016B800151216E7901A0378807B0A1216E6A3081B
:1016C800DBF9901A0F788C7B191216E6A308DBF960
:1016D800121734121712901A2822E493F622E643BE
:1016E8008F01538FFD75EF0275B7A575B7F1F053EC
:1016F8008FFE22438F02438F0175EF0275B7A575E0
:10170800B7F1901A0DF0538FFC22901A0D74A5D1E1
:10171800E7901A0E745AD1E7227A3079D07820905F
:101728001A40D1E2E520F709A3DAF7227A3079D016
:10173800901A40E7D1E709A3DAF922AB74A875BB80
:1017480001027980BB02027981BB03027982BB0462
:10175800027994BB05027983BB06027986BB07022E
:101768007992BB08027987BB0902799CBB0A027986
:1017780088BB0B027989E8F7227C0512055FDCFB40
:1017880022C2AF12056F12057612057D120584126A
:10179800055012056F12057612057D120584120593
:1017A8005012056F12057612057D120584D2AF22FC
:1017B800C2AF12058412057D12057612056F120557
:1017C8005012058412057D12057612056F12055018
:1017D80012058412057D12057612056FD2AF22AE6E
:1017E80074AF75C2AF12056F12056F12056F12053F
:1017F80050DEF2120584120550DFF8D2AF2212171C
:101808008912178112178175740175750175760033
:101818001217E77C05AD5C12055FC3ED955C70F5AA
:10182800C3E55C9401400AC3E55C94FF40370218A5
:101838004A1217431216A0121789C2AF75EF121277
:101848001781DCD10576C3E5769403500280C11276
:1018580017810575E5741490009F93F808C3E57522
:0E18680098500280A81217811217810574C3D0
:10187600E574940C50028094120FE91216A0C2AFC0
:0618860075EF121217813C
:0319FD000211557F
:101A00000E061507070104FFFF0A020101A55A018E
:101A100000B4FFFFFF03FF01FF25D078C804FF01DA
:091A200000FF0A010100FF00FFB4
:101A400023585032354123202020202020202020E0
:101A500023424C48454C4923463333302320202031
:101A60002020202020202020202020202020202076
:101C0000C2AFC2D353D9BF7581C043B20343FF8073
:101C1000752438752503B1C975EF0275E24043F1AB
:101C20008053A47F75D4FFD2877DFA780379E67C50
:101C300010752200752300901DD67B0675249875BB
:101C400025013087028142208708D8FBD9F9DCF7CB
:101C500081B4308708D8FBD9F9DCF781B4B189E4C5
:101C600093A3C39A6004DDC381B4DBDBB17B600264
:101C7000812B7B08E493FAA3B15CDBF87A30B15C8A
:101C8000752200752300B17BEAFCEBFDC3ED94FEE9
:101C9000400EB17B8A278B28ED30E0048A828B834B
:101CA000B17B7AC270D8C3ED94FE601350CEBD00F4
:101CB00025EC60097520007521FF0200008100A855
:101CC00027A9280809D804D90281D3B17FEA89AAB3
:101CD000F281C50D81A0C3ED94035049EDA2E092BD
:101CE000007AC5C3E5829400E583941C50902000DF
:101CF00010438F02438F0175B7A575B7F1F030001F
:101D00001FA827A9280809438F01538FFDD804D99C
:101D100002A12089AAE275B7A575B7F1F0A3A10DBC
:101D2000538FFC817C7AC1BD030CE493A3FAB140CC
:101D3000DCF8B138817C817EAA22AB23B15CEBFA5E
:101D4000EA6222752608C3E52313F523E52213F57D
:101D50002250066323A0632201D526EAB1C9B1C986
:101D600075260AEAF4200102D287300102C287B147
:101D7000C9C3134002C201D526EB22B17FEAFB2082
:101D80008702A17F308702A184752608AE24AF2583
:101D9000C3EF13FFEE13FEB1CDB1C9C3EA13308711
:101DA000024480FA30E703632201C3E52313F523DD
:101DB000E52213F52250066323A0632201D526D91C
:101DC000E52265236523F52222AE24AF250E0FDE22
:101DD000FEDFFCD20122424C48656C693437316326
:041DE000F3300601D5
:00000001FF
